Archive member included because of file (symbol)

c:/program files/yagarto/bin/../lib/gcc/arm-elf/4.3.3\libgcc.a(_udivsi3.o)
                              ../common/src/rprintf.o (__udivsi3)
c:/program files/yagarto/bin/../lib/gcc/arm-elf/4.3.3\libgcc.a(_umodsi3.o)
                              ../common/src/rprintf.o (__umodsi3)
c:/program files/yagarto/bin/../lib/gcc/arm-elf/4.3.3\libgcc.a(_dvmd_tls.o)
                              c:/program files/yagarto/bin/../lib/gcc/arm-elf/4.3.3\libgcc.a(_udivsi3.o) (__div0)

Allocating common symbols
Common symbol       size              file

sp                  0x4               DAC.o
s                   0x14              DAC.o

Memory Configuration

Name             Origin             Length             Attributes
flash            0x00000000         0x00080000
ram_isp_low      0x40000120         0x000000df         a
ram              0x40000200         0x00007f01
ram_isp_high     0x40007fe0         0x00000020         a
ram_usb_dma      0x7fd00000         0x00002000
*default*        0x00000000         0xffffffff

Linker script and memory map

LOAD ../common/src/crt.o
LOAD ../common/src/startup.o
LOAD ../common/src/TFT018.o
LOAD ../common/src/rprintf.o
LOAD DAC.o
START GROUP
LOAD c:/program files/yagarto/bin/../lib/gcc/arm-elf/4.3.3\libgcc.a
LOAD c:/program files/yagarto/bin/../lib/gcc/arm-elf/4.3.3/../../../../arm-elf/lib\libc.a
END GROUP
                0x40007edc                _stack_end = 0x40007edc
                0x00000000                . = 0x0

startup
 *(.startup)

.text           0x00000000     0x23c4
 *(.text)
 .text          0x00000000       0xd8 ../common/src/crt.o
                0x00000000                _startup
                0x00000040                Reset_Handler
 .text          0x000000d8       0x84 ../common/src/startup.o
                0x000000e4                UNDEF_Routine
                0x000000e0                SWI_Routine
                0x000000dc                FIQ_Routine
                0x000000d8                IRQ_Routine
                0x000000e8                Initialize
 .text          0x0000015c      0xaf4 ../common/src/TFT018.o
                0x00000280                LCD_Reg_Set
                0x00000454                LCD_SetArea
                0x00000a74                LCD_PutString
                0x0000059c                LCD_Clear_Screen
                0x000004b4                LCD_Rectangle
                0x00000b18                LCD_BMP
                0x00000798                LCD_PutChar8x8
                0x0000015c                BacklightOn
                0x000005c4                LCD_SetPixel
                0x00000218                LCD_Bus_Write_Data
                0x00000300                LCD_Init
                0x000008c8                LCD_PutChar
                0x000001bc                LCD_Bus_Initial
                0x00000664                LCD_PutChar8x16
                0x00000c18                LCD_Bus_Read_Pixel
                0x0000025c                LCD_Bus_Read_Byte
                0x000001b8                Delay1Ms
                0x000001ec                LCD_Bus_Write_Byte
                0x00000900                PutGB1616
 .text          0x00000c50      0x258 ../common/src/rprintf.o
                0x00000c50                rprintf_devopen
                0x00000c94                rprintf
 .text          0x00000ea8       0xe8 DAC.o
                0x00000ec0                input_str
                0x00000ea8                DACInit
                0x00000ee4                main
 .text          0x00000f90      0x110 c:/program files/yagarto/bin/../lib/gcc/arm-elf/4.3.3\libgcc.a(_udivsi3.o)
                0x00000f90                __udivsi3
                0x00000f90                __aeabi_uidiv
                0x00001088                __aeabi_uidivmod
 .text          0x000010a0       0xcc c:/program files/yagarto/bin/../lib/gcc/arm-elf/4.3.3\libgcc.a(_umodsi3.o)
                0x000010a0                __umodsi3
 .text          0x0000116c        0x4 c:/program files/yagarto/bin/../lib/gcc/arm-elf/4.3.3\libgcc.a(_dvmd_tls.o)
                0x0000116c                __aeabi_ldiv0
                0x0000116c                __div0
                0x0000116c                __aeabi_idiv0
 *(.rodata)
 .rodata        0x00001170     0x1248 ../common/src/TFT018.o
                0x00002178                codeGB_16
                0x00001970                Font8x8
                0x00001170                Font8x16
 *(.rodata*)
 .rodata.str1.1
                0x000023b8        0xc DAC.o
 *(.glue_7)
 .glue_7        0x000023c4        0x0 ../common/src/crt.o
 .glue_7        0x000023c4        0x0 ../common/src/startup.o
 .glue_7        0x000023c4        0x0 ../common/src/TFT018.o
 .glue_7        0x000023c4        0x0 ../common/src/rprintf.o
 .glue_7        0x000023c4        0x0 DAC.o
 .glue_7        0x000023c4        0x0 c:/program files/yagarto/bin/../lib/gcc/arm-elf/4.3.3\libgcc.a(_udivsi3.o)
 .glue_7        0x000023c4        0x0 c:/program files/yagarto/bin/../lib/gcc/arm-elf/4.3.3\libgcc.a(_umodsi3.o)
 .glue_7        0x000023c4        0x0 c:/program files/yagarto/bin/../lib/gcc/arm-elf/4.3.3\libgcc.a(_dvmd_tls.o)
 *(.glue_7t)
 .glue_7t       0x000023c4        0x0 ../common/src/crt.o
 .glue_7t       0x000023c4        0x0 ../common/src/startup.o
 .glue_7t       0x000023c4        0x0 ../common/src/TFT018.o
 .glue_7t       0x000023c4        0x0 ../common/src/rprintf.o
 .glue_7t       0x000023c4        0x0 DAC.o
 .glue_7t       0x000023c4        0x0 c:/program files/yagarto/bin/../lib/gcc/arm-elf/4.3.3\libgcc.a(_udivsi3.o)
 .glue_7t       0x000023c4        0x0 c:/program files/yagarto/bin/../lib/gcc/arm-elf/4.3.3\libgcc.a(_umodsi3.o)
 .glue_7t       0x000023c4        0x0 c:/program files/yagarto/bin/../lib/gcc/arm-elf/4.3.3\libgcc.a(_dvmd_tls.o)
                0x000023c4                _etext = .

.vfp11_veneer   0x40000120        0x0
 .vfp11_veneer  0x40000120        0x0 ../common/src/crt.o
 .vfp11_veneer  0x40000120        0x0 ../common/src/startup.o
 .vfp11_veneer  0x40000120        0x0 ../common/src/TFT018.o
 .vfp11_veneer  0x40000120        0x0 ../common/src/rprintf.o
 .vfp11_veneer  0x40000120        0x0 DAC.o
 .vfp11_veneer  0x40000120        0x0 c:/program files/yagarto/bin/../lib/gcc/arm-elf/4.3.3\libgcc.a(_udivsi3.o)
 .vfp11_veneer  0x40000120        0x0 c:/program files/yagarto/bin/../lib/gcc/arm-elf/4.3.3\libgcc.a(_umodsi3.o)
 .vfp11_veneer  0x40000120        0x0 c:/program files/yagarto/bin/../lib/gcc/arm-elf/4.3.3\libgcc.a(_dvmd_tls.o)

.v4_bx          0x40000120        0x0
 .v4_bx         0x40000120        0x0 ../common/src/crt.o
 .v4_bx         0x40000120        0x0 ../common/src/startup.o
 .v4_bx         0x40000120        0x0 ../common/src/TFT018.o
 .v4_bx         0x40000120        0x0 ../common/src/rprintf.o
 .v4_bx         0x40000120        0x0 DAC.o
 .v4_bx         0x40000120        0x0 c:/program files/yagarto/bin/../lib/gcc/arm-elf/4.3.3\libgcc.a(_udivsi3.o)
 .v4_bx         0x40000120        0x0 c:/program files/yagarto/bin/../lib/gcc/arm-elf/4.3.3\libgcc.a(_umodsi3.o)
 .v4_bx         0x40000120        0x0 c:/program files/yagarto/bin/../lib/gcc/arm-elf/4.3.3\libgcc.a(_dvmd_tls.o)

.data           0x40000200        0x0 load address 0x000023c4
                0x40000200                _data = .
 *(.data)
 .data          0x40000200        0x0 ../common/src/crt.o
 .data          0x40000200        0x0 ../common/src/startup.o
 .data          0x40000200        0x0 ../common/src/TFT018.o
 .data          0x40000200        0x0 ../common/src/rprintf.o
 .data          0x40000200        0x0 DAC.o
 .data          0x40000200        0x0 c:/program files/yagarto/bin/../lib/gcc/arm-elf/4.3.3\libgcc.a(_udivsi3.o)
 .data          0x40000200        0x0 c:/program files/yagarto/bin/../lib/gcc/arm-elf/4.3.3\libgcc.a(_umodsi3.o)
 .data          0x40000200        0x0 c:/program files/yagarto/bin/../lib/gcc/arm-elf/4.3.3\libgcc.a(_dvmd_tls.o)
                0x40000200                _edata = .

.bss            0x40000200       0x20
                0x40000200                _bss_start = .
 *(.bss)
 .bss           0x40000200        0x0 ../common/src/crt.o
 .bss           0x40000200        0x0 ../common/src/startup.o
 .bss           0x40000200        0x1 ../common/src/TFT018.o
                0x40000200                Font
 *fill*         0x40000201        0x3 00
 .bss           0x40000204        0x4 ../common/src/rprintf.o
 .bss           0x40000208        0x0 DAC.o
 .bss           0x40000208        0x0 c:/program files/yagarto/bin/../lib/gcc/arm-elf/4.3.3\libgcc.a(_udivsi3.o)
 .bss           0x40000208        0x0 c:/program files/yagarto/bin/../lib/gcc/arm-elf/4.3.3\libgcc.a(_umodsi3.o)
 .bss           0x40000208        0x0 c:/program files/yagarto/bin/../lib/gcc/arm-elf/4.3.3\libgcc.a(_dvmd_tls.o)
 COMMON         0x40000208       0x18 DAC.o
                0x40000208                sp
                0x4000020c                s
                0x40000220                . = ALIGN (0x4)
                0x40000220                _bss_end = .
                0x40000220                _end = .
OUTPUT(DAC.elf elf32-littlearm)

.ARM.attributes
                0x00000000       0x10
 .ARM.attributes
                0x00000000       0x10 ../common/src/crt.o
 .ARM.attributes
                0x00000010       0x10 ../common/src/startup.o
 .ARM.attributes
                0x00000020       0x10 ../common/src/TFT018.o
 .ARM.attributes
                0x00000030       0x10 ../common/src/rprintf.o
 .ARM.attributes
                0x00000040       0x10 DAC.o
 .ARM.attributes
                0x00000050       0x10 c:/program files/yagarto/bin/../lib/gcc/arm-elf/4.3.3\libgcc.a(_udivsi3.o)
 .ARM.attributes
                0x00000060       0x10 c:/program files/yagarto/bin/../lib/gcc/arm-elf/4.3.3\libgcc.a(_umodsi3.o)
 .ARM.attributes
                0x00000070       0x10 c:/program files/yagarto/bin/../lib/gcc/arm-elf/4.3.3\libgcc.a(_dvmd_tls.o)

.debug_abbrev   0x00000000      0x589
 .debug_abbrev  0x00000000       0x69 ../common/src/startup.o
 .debug_abbrev  0x00000069      0x2bd ../common/src/TFT018.o
 .debug_abbrev  0x00000326      0x140 ../common/src/rprintf.o
 .debug_abbrev  0x00000466       0xe7 DAC.o
 .debug_abbrev  0x0000054d       0x14 c:/program files/yagarto/bin/../lib/gcc/arm-elf/4.3.3\libgcc.a(_udivsi3.o)
 .debug_abbrev  0x00000561       0x14 c:/program files/yagarto/bin/../lib/gcc/arm-elf/4.3.3\libgcc.a(_umodsi3.o)
 .debug_abbrev  0x00000575       0x14 c:/program files/yagarto/bin/../lib/gcc/arm-elf/4.3.3\libgcc.a(_dvmd_tls.o)

.debug_info     0x00000000     0x1019
 .debug_info    0x00000000       0xb4 ../common/src/startup.o
 .debug_info    0x000000b4      0xa85 ../common/src/TFT018.o
 .debug_info    0x00000b39      0x207 ../common/src/rprintf.o
 .debug_info    0x00000d40      0x11d DAC.o
 .debug_info    0x00000e5d       0x94 c:/program files/yagarto/bin/../lib/gcc/arm-elf/4.3.3\libgcc.a(_udivsi3.o)
 .debug_info    0x00000ef1       0x94 c:/program files/yagarto/bin/../lib/gcc/arm-elf/4.3.3\libgcc.a(_umodsi3.o)
 .debug_info    0x00000f85       0x94 c:/program files/yagarto/bin/../lib/gcc/arm-elf/4.3.3\libgcc.a(_dvmd_tls.o)

.debug_line     0x00000000      0x667
 .debug_line    0x00000000       0x77 ../common/src/startup.o
 .debug_line    0x00000077      0x32c ../common/src/TFT018.o
 .debug_line    0x000003a3       0xd6 ../common/src/rprintf.o
 .debug_line    0x00000479       0x6f DAC.o
 .debug_line    0x000004e8       0x96 c:/program files/yagarto/bin/../lib/gcc/arm-elf/4.3.3\libgcc.a(_udivsi3.o)
 .debug_line    0x0000057e       0x7f c:/program files/yagarto/bin/../lib/gcc/arm-elf/4.3.3\libgcc.a(_umodsi3.o)
 .debug_line    0x000005fd       0x6a c:/program files/yagarto/bin/../lib/gcc/arm-elf/4.3.3\libgcc.a(_dvmd_tls.o)

.debug_frame    0x00000000      0x350
 .debug_frame   0x00000000       0x60 ../common/src/startup.o
 .debug_frame   0x00000060      0x1e0 ../common/src/TFT018.o
 .debug_frame   0x00000240       0x6c ../common/src/rprintf.o
 .debug_frame   0x000002ac       0x54 DAC.o
 .debug_frame   0x00000300       0x28 c:/program files/yagarto/bin/../lib/gcc/arm-elf/4.3.3\libgcc.a(_udivsi3.o)
 .debug_frame   0x00000328       0x28 c:/program files/yagarto/bin/../lib/gcc/arm-elf/4.3.3\libgcc.a(_umodsi3.o)

.debug_pubnames
                0x00000000      0x26d
 .debug_pubnames
                0x00000000       0x63 ../common/src/startup.o
 .debug_pubnames
                0x00000063      0x196 ../common/src/TFT018.o
 .debug_pubnames
                0x000001f9       0x32 ../common/src/rprintf.o
 .debug_pubnames
                0x0000022b       0x42 DAC.o

.debug_aranges  0x00000000       0xe0
 .debug_aranges
                0x00000000       0x20 ../common/src/startup.o
 .debug_aranges
                0x00000020       0x20 ../common/src/TFT018.o
 .debug_aranges
                0x00000040       0x20 ../common/src/rprintf.o
 .debug_aranges
                0x00000060       0x20 DAC.o
 .debug_aranges
                0x00000080       0x20 c:/program files/yagarto/bin/../lib/gcc/arm-elf/4.3.3\libgcc.a(_udivsi3.o)
 .debug_aranges
                0x000000a0       0x20 c:/program files/yagarto/bin/../lib/gcc/arm-elf/4.3.3\libgcc.a(_umodsi3.o)
 .debug_aranges
                0x000000c0       0x20 c:/program files/yagarto/bin/../lib/gcc/arm-elf/4.3.3\libgcc.a(_dvmd_tls.o)

.debug_ranges   0x00000000      0x7a8
 .debug_ranges  0x00000000       0x30 ../common/src/startup.o
 .debug_ranges  0x00000030      0x760 ../common/src/TFT018.o
 .debug_ranges  0x00000790       0x18 ../common/src/rprintf.o

.debug_str      0x00000000      0x313
 .debug_str     0x00000000       0x89 ../common/src/startup.o
 .debug_str     0x00000089      0x1af ../common/src/TFT018.o
                                0x1f5 (size before relaxing)
 .debug_str     0x00000238       0xbe ../common/src/rprintf.o
                                0x17e (size before relaxing)
 .debug_str     0x000002f6       0x1d DAC.o
                                 0xae (size before relaxing)

.comment        0x00000000       0x48
 .comment       0x00000000       0x12 ../common/src/startup.o
 .comment       0x00000012       0x12 ../common/src/TFT018.o
 .comment       0x00000024       0x12 ../common/src/rprintf.o
 .comment       0x00000036       0x12 DAC.o

.debug_loc      0x00000000      0xb4f
 .debug_loc     0x00000000      0x927 ../common/src/TFT018.o
 .debug_loc     0x00000927      0x1ea ../common/src/rprintf.o
 .debug_loc     0x00000b11       0x3e DAC.o
